:10000000F4288030A100FE308F2001308F20753021
:10001000A9003030C028A101A117B100FE308F2007
:1000200031088F28A01125080319A0150530A40058
:100030002730AB00103028200330AB00E8302820F8
:10004000AB0164302820AB010A3028202C082F286F
:10005000AA002D08A9002C08A800D4202808A80070
:10006000A4030319A0112508031939282402031831
:1000700040282808031DA011A0194028303E8F28D1
:100080000800AF0087120712831687120712F0309C
:10009000870583122F08A0186B283E30A9008030F6
:1000A000C0203330AE0080201330A9008830C0203B
:1000B00080206430BF2080206430BF202230AE001A
:1000C000802028306A200C306A2006306A20A01474
:1000D0002F086B282014AE00201C79280712033C3F
:1000E000031C7E287E200730A900D030C0200314D6
:1000F00008002014FE3C03198D280716AE0E201CA4
:1001000020108716F03087052E080F3987048712D4
:10011000AE0E201880283230BF202F08F028A11BF7
:10012000412808000739AE000310AE0DAE0D30387F
:1001300083169F0083121F08E3392E0401389F00A5
:100140003230BF209F149F18A3281E08B5008316C5
:100150001E088312B400F0288001840AFF3E031DAC
:10016000AC28F028AB01AA00FF30AA07031CAB079C
:10017000031CF0280330A900DF30C020B428A901F7
:10018000E83EA800A909FC30031CC928A8070318E9
:10019000C628A8070000A90FC6282818CF28A81C21
:1001A000D3280000D3280800AD01AC011030AE0008
:1001B000290DAC0DAD0D2A08AC022B08031C2B0F2A
:1001C000AD020318EA282A08AC072B0803182B0FE6
:1001D000AD070310A80DA90DAE0BD8282808F028EC
:1001E0008313831203130800A00185018701CE3019
:1001F00083168500FF308700803083129F008316AE
:100200009F0106309100073083129900203084004E
:100210004030AC200130AB00F430B32001208030FE
:10022000A10081300B20413041206E3041206130EF
:1002300041206C3041206F30412041206730412007
:100240003A3041208030A100C0300B205030412096
:100250006F304120743041206D30412065304120A5
:100260007430412065304120723041203A304120C5
:100270000130DD0005305D02031846290130850696
:10028000AB002C30B320DD0A031D3A290230922046
:10029000A6003508A70003105C0D363E8400260832
:1002A0008000840A270880000E305C0203185A2957
:1002B000DC0AD829DC01D501D401DD010F305D0253
:1002C0000318742903105D0D363E84000008A60053
:1002D000840A0008A7002608D40727080318013E4F
:1002E000D507DD0A031D5E295508A9005408A8009A
:1002F000AB010F30AA00D420D4002908D50001306A
:100300009220D6003508D7008030A100CA300B20DB
:100310000430A5005708AD005608AC00122001308B
:100320005702C23003195602031897299E298512D5
:100330000512D901D801FA30B2207F298030A100FE
:100340008A300B200430A5005508AD005408AC00DD
:10035000122055085702031CB329031DD329540842
:1003600056020318D329D80A0319D90A0D305902A5
:10037000031CC629031DC029AD305802031CC62921
:1003800005160B30D900EA30D800C729051205142C
:100390005808143A5904031DD22985160516C83089
:1003A000B2200512D829D901D801851205100512ED
:0803B0000530B2204629DB29CB
:02400E00A43FCD
:00000001FF
